:1000000056C0BAC16FC06EC06DC06CC06BC06AC054
:1000100069C068C067C066C065C064C063C062C0B4
:1000200061C060C05FC0040309040A0359004300B3
:100030004900540010034800490044006100730067
:10004000700078000A0330003000300030001201E8
:10005000100100000008C016DF05000101020301C5
:1000600009021B00010100803209040000000300A6
:1000700000000921010100012233000600FF0901EF
:10008000A101150026FF007508850195060900B23B
:1000900002018502951E0900B20201850395260919
:1000A00000B20201850495040900B20201C01124C6
:1000B0001FBECFE5D4E0DEBFCDBF10E0A0E6B0E0CC
:1000C000EEE2F8E002C005900D92A236B107D9F732
:1000D00010E0A2E6B0E001C01D92A53BB107E1F738
:1000E0008BD3A3C38DCF85B78C6085BF8BB780645E
:1000F0008BBF08951F93CF93DF9360919B00635054
:1001000067FDC6C080919800CCE0D0E0C81BD10943
:10011000C156DF4F809197008D3209F0A3C068303F
:1001200009F0B0C083EC80938B008AE58093600077
:10013000109262008881807639F0CE014AD2282F51
:100140008F3F09F47EC084C09A8110929400898107
:10015000882321F41092950022E06CC0853019F4B8
:1001600090939C0066C0863009F054C08B8181302A
:1001700041F48EE490E090939A008093990022E1FC
:1001800045C0823041F480E690E090939A008093DD
:1001900099002BE13BC0833021F58A81882341F40B
:1001A00086E290E090939A008093990024E02EC01C
:1001B000813019F48AE290E00EC0823041F484E389
:1001C00090E090939A008093990020E11FC08330C3
:1001D000E1F484E490E090939A00809399002AE0FF
:1001E00015C0813241F482E790E090939A008093A9
:1001F000990029E00BC0823241F48BE790E09093A4
:100200009A008093990023E301C020E080E480936A
:1002100062001EC0883021F421E08EE990E00CC01D
:10022000893019F490939E0004C08A3011F421E0C3
:1002300001C020E084E990E090939A0080939900B7
:1002400007C0888187FD2E8180E88093620006C008
:100250008F81882319F48E81821708F0822F809372
:10026000610010C08091620087FF0CC0CE01A4D253
:100270008F3F21F48EE18093600004C0882311F049
:100280001092610080919B00181614F410929B004C
:100290008091600084FF49C0809161008F3F09F424
:1002A00044C0182F893008F018E0811B809361004A
:1002B00080918B0098E8892780938B00112341F16E
:1002C0002091990030919A008091620086FF0DC0C4
:1002D000ACE8B0E080E090E0F901E80FF91FE491AC
:1002E000ED9301961817C1F708C0912FD901ECE8DA
:1002F000F0E08D9181939150E1F71150812F90E0C2
:100300001F5F0196820F931F90939A00809399002C
:100310008CE890E0612F2CD0612F6C5F6C3019F06D
:100320008FEF809361006093600094E186B38370E7
:1003300031F49150D9F710929C0010929600DF9101
:10034000CF911F910895A82FB92F80E090E041E050
:1003500050EA609530E009C02D91822797958795E6
:1003600010F084279527305EC8F36F5FA8F30895D7
:10037000EADF8D939D930895CF93CFB7CF93C39525
:10038000B09BE9F7B09B09C0B09B07C0B09B05C00C
:10039000B09B03C0B09B01C0A1C0DF93C091980087
:1003A000DD27C156DF4FB09B02C0DF91EBCF2F930B
:1003B0000F931F9306B32FEF00FB20F94F933F934A
:1003C00016B34FEF012700FB21F93BE031C04E7F10
:1003D000012F16B3216028C0102F4D7F226000002E
:1003E00006B329C04B7F2460012F000016B32BC039
:1003F00016B3477F28602AC04F7E06B320612CC009
:100400004F7D16B320622FC04F7B06B3206432C0ED
:10041000422706B349934FEF0000102710FB20F945
:1004200016B31370C9F1297F91F2012700FB21F95E
:1004300006B3237F89F2315058F1102710FB22F9BF
:1004400016B3277E79F2012700FB23F92F7C81F276
:1004500006B3102710FB24F92F7971F200C016B3F0
:10046000012700FB25F92F7359F200C006B31027AE
:1004700010FB26F9223040F200C016B3012700FB22
:1004800027F9243028F64F77206816B30000F9CFFB
:1004900010E41ABF002717C03B503195C31BD04052
:1004A00010E41ABF0881033CE9F00B34D9F0209125
:1004B00096001981110F1213EDCF093641F10D325B
:1004C00011F0013E39F700939D003F914F911F912C
:1004D0000F912F91DF91CAB7C6FD51CFCF91CFBFFA
:1004E000CF91189520919D00222379F310919B00C4
:1004F000112311F5343012F130939B0020939700B3
:10050000109198003BE0311B3093980017C0009188
:100510009B0001308CF40AE53091600034FD10C07E
:1005200000936000CBE8D0E00FC02795A8F45150AD
:10053000A9F4220F0000F9CF4AE503C042ED01C043
:10054000432FC4E1D0E032E017B31360C09A17BB69
:1005500008B320E413E05F93012756E008BB27951A
:1005600020F4515021F4220FF9CF012756E000006A
:100570003B5A08BBD0F2279528F4515029F4220F9A
:100580000000F9CF012756E0279508BB20F4515011
:1005900021F4220FF9CF012756E02991332308BB1C
:1005A00021F60C7F10919C00110FC651D04008BB62
:1005B00011F01093960010E41ABF016017B31C7F6E
:1005C000402F4C7F5F9100C000C008BB17BB48BBE9
:1005D0007CCFDC0111969C9111978C9180768032B2
:1005E000F1F49130A9F412962C91129720936300A4
:1005F00083E690E090939A0080939900243029F448
:10060000E72DF0E080818093640016968C91089528
:10061000993029F4442416965C908FEF089580E079
:100620000895CF93DF93909164002091650085E554
:1006300080936400923019F5AA2011F48AEB1CC053
:100640008091660084FF04C08FE084BB8BE012C001
:1006500087FF05C0AF9A84E6E2D0AF980CC08FED5B
:1006600084BBAC98AF9886E0DAD0AC9A84E6D7D059
:1006700085B38D7E85BB8AEA809364009AC0392F4A
:100680003E7F303179F4E4E6F0E091E581819DB977
:100690008FB9779BFECF8FB1819380E0E836F80762
:1006A000A9F787C0943131F4622E70906600809073
:1006B00067007FC0892F887F803209F056C08FEF96
:1006C00080939B00792F91FF04C030E4632E772440
:1006D0008824A4E6B0E0FD01422F50E0EA01CA0FF1
:1006E000DB1F31E52AC0962D3DB96FB8779BFECF51
:1006F0008FB1682D3DB98FB8779BFECF8FB1272D75
:100700003DB97FB8779BFECF8FB182813DB98FB95C
:10071000779BFECF8FB18083892F887851F0822F0D
:100720008F5F782E11F4862E839427EF622E692234
:1007300003C088E0682E692A3196EC17FD0799F608
:1007400072FF10C0FA01EA59FF4F91E580819DB90F
:100750008FB9779BFECF8FB18D93319680E0A8360D
:10076000B807A1F710929B0024C09C3311F4922E7D
:1007700020C03E33F1F4A0916600B09167009F3332
:1007800061F4922FC4E6D0E0FD0102C0819189930B
:100790008E2F8A1B8917D0F30CC02091680090918E
:1007A0006900992329F08C919823922B9C9301C086
:1007B0002C93DF91CF910895582F292F852D561610
:1007C00008F4652D482F461B542E852F922F9C012F
:1007D000D90107C0E42DF0E0ED59FF4F9D919083C2
:1007E00043948A2F851B8617A8F3442311F080E0D9
:1007F000089517DF81E00895992403C088EC0FD095
:10080000939485E98915D0F7959A8CEF81BB8BE09D
:1008100085BB8FE084BB67DC78946CDCFECF98E20C
:0E0820009150F1F78150D9F70895F894FFCF69
:02082E005AFF6F
:00000001FF
